:10000000F9C0000013C1000011C100000FC10000C1
:100010000DC100000BC1000009C1000007C10000B4
:1000200005C1000003C1000001C100000C943E1294
:10003000FDC00000FBC00000F9C000006FC7000059
:10004000F5C00000F3C00000F1C00000A3C1000033
:10005000EDC00000EBC00000E9C00000E7C00000F8
:10006000E5C00000E3C00000E1C00000DFC0000008
:10007000DDC0000018034100560052004900530043
:10008000500020006D006B004900490000000C0387
:10009000410054004D0045004C00000004030904D9
:1000A00012011001FF000010EB0304210002010205
:1000B00003014000410142430309000A000A000B0A
:1000C000000C000D000D000E000F001000100012BB
:1000D0000013001300140016001600180019001A6F
:1000E000001C001D001F0020002200230025002707
:1000F0000029002B002E0030003200340037003A77
:10010000003D004000430046004A004E00520055AA
:10011000005A005E00630068006D00730078007E86
:100120000084008B0091009900A000A900B100B9E3
:1001300000C300CC00D600E100EC00F70004011180
:10014000011E012D013B014B015B016C017D019101
:1001500001A501BA01CF01E601FE01160231024CF0
:10016000026A028802A802CA02ED02110338036083
:10017000038B03B803E70318044B048104B904F5A7
:100180000434057505B90501064E069D06EF0648BF
:1001900007A30704086508D0084009B6092B0AAB75
:1001A0000A300BC30B510CEE0C8F0D400EF60EAF48
:1001B0000F681047111412F512ED13E214F015F93F
:1001C000161B185C19911AE51B251D831E0320AB15
:1001D00021302332250F27F128F82A1A2D492FA183
:1001E000311434A1364539173C1A3F34426045DF9B
:1001F00048704C0011241FBECFEFD2E0DEBFCDBF50
:1002000011E0A0E0B1E0E8E5F8E202C005900D924F
:10021000A23AB107D9F721E0A2EAB1E001C01D92EC
:10022000A53BB207E1F74ED00C942A14E9CE95B164
:100230009F71982B95B9089584B7877F84BF88E113
:100240000FB6F89480936000109260000FBE90E0AB
:1002500080E80FB6F89480936100909361000FBE20
:1002600084B1806E84B985B18F7185B90C942F12D9
:1002700080ECDDCF80E4DBCFCF9342E360E882E027
:100280000E949711C82F42E361E883E00E94971112
:10029000882321F0CC2311F080E801C080E4CF91C5
:1002A000C6CF8EB3843069F4D3D182E08093E90065
:1002B0008091E80082FF05C080ECB9DF88D080E83B
:1002C000B6CF0895B9DF7BD080E4B1DF7894489B46
:1002D00002C090E001C090E285B18F7D892B85B985
:1002E000E0DF0E94F513F3CF00C0D9011C92292F43
:1002F00033272230310541F02330310561F02130C0
:10030000310509F439C03DC082E08C93E0E2F0E0B1
:100310008EE191E03AC099278130910589F01CF473
:10032000892B39F02EC08230910589F0039749F569
:1003300015C0ECE9F0E0E491F0E08CE990E025C034
:10034000EEE8F0E0E491F0E08EE890E01EC0E4E733
:10035000F0E0E491F0E084E790E017C0E091000164
:10036000F0E083E390E090930F0180930E0182E030
:100370008C9380E091E009C0E2E1F0E080EA90E057
:1003800004C0E0E0F0E080E090E0DA018D939C931F
:10039000CF01089578941F920F920FB60F921124F7
:1003A0008F938AB5882321F08AB581508ABD01C018
:1003B00015BC8F910F900FBE0F901F9018958BE971
:1003C00087BD82E084BD80936E0027D1D5C50F9391
:1003D0001F93CF93DF931F92CDB7DEB71091F1003B
:1003E00084E68ABD85E085BD143109F4C4C000F5FA
:1003F0001A3009F4A7C068F4143038F4123008F049
:1004000050C0113009F0CFC02FC0163009F0CBC05A
:1004100073C0113109F4AAC020F4103109F0C3C02F
:10042000A3C0123109F4AAC0133109F0BCC0A0C0A6
:10043000193109F4A8C060F4163109F49CC008F41D
:1004400097C0173109F49FC0183109F0ACC098C0AB
:100450001D3109F49BC008F493C0103509F49AC00B
:10046000113509F0A0C094C08091E8008B7780938B
:10047000E80083E08093E9008091EC008160809344
:10048000EC001093F1001092F1008AE08093F100EB
:1004900040E050E06AE070E087E991E00E947A0F66
:1004A00098C00091F100123011F46091F100809138
:1004B000E8008B778093E80083E08093E9008091E7
:1004C000EC0081608093EC001093F100802F698331
:1004D000C0D06981123039F481FF0CC01092F10054
:1004E000802FC7D076C080FF05C01092F100802F0A
:1004F000B8D06DC080EC6BC040E050E064E070E0CC
:1005000086EA91E00E9416108091E8008B77809334
:10051000E80083E08093E9008091EC0081608093A3
:10052000EC008091A6019091A701A091A801B09143
:10053000A901B7FF03C081E08093A50186E0809305
:10054000F1000FC08091E8008B778093E80083E092
:100550008093E9008091EC0081608093EC0010931F
:10056000F1001092F10035C055D438C01FD436C008
:10057000812FC2D033C0812FFBD130C0CAD32EC04F
:10058000812F94D22BC0812FECD228C030D326C02B
:100590003AD724C068D722C08091E8008B77809337
:1005A000E8000E94CA118091F2008034A9F3809182
:1005B000E8008B778093E80083E08093E9008091E6
:1005C000EC0081608093EC001093F10089EC809343
:1005D000F1008091E8008E778093E80015BC0E94BE
:1005E000CA1182E08093E9008091EC008E7F8093B5
:1005F000EC000F90DF91CF911F910F910895EEE3E2
:10060000F1E09081891739F0339691E0EC35F907E4
:10061000C1F7E0E0F0E0CF010895CF93DF9380E0F1
:1006200090E00E941014D82F81E090E00E941014F6
:10063000C82FDF3F21F08EE9E2DFFC01D283CF3FFC
:1006400021F088E9DCDFFC01C283DF91CF910895BE
:100650000895D5DF009719F0FC018181089580E0AD
:100660000895CDDF009719F0FC018281089580E0A4
:1006700008951F93CF93DF931F92CDB7DEB7182F46
:100680006983BDDF6981009789F0FC0162831E39AF
:1006900019F480E090E004C0183941F481E090E062
:1006A0000F90DF91CF911F910C9418140F90DF9150
:1006B000CF911F91089590915C01992329F08EBDEF
:1006C0000DB407FEFDCF0895BEC490915C0199233F
:1006D00031F08EBD0DB407FEFDCF8EB50895B3C4C5
:1006E00080915C01882331F01EBC0DB407FEFDCF64
:1006F0008EB5089580E0A7C45F926F927F928F922B
:100700009F92AF92BF92CF92DF92EF92FF920F93A0
:100710001F93CF93DF93CDB7DEB7CA50D1400FB64A
:10072000F894DEBF0FBECDBF182F40E050E069E067
:1007300070E0CE0101960E94C80F6A8179817A83A8
:100740006983613081E0780788F08091E8008B77D9
:100750008093E80083E08093E9008091EC00816061
:100760008093EC001093F10080ECE4C040E050E096
:10077000CE010A960E94C80F89819A810A968F73CA
:100780009927892B39F48091E8008B778093E800D2
:100790000E94CA118091E8008B778093E80083E083
:1007A0008093E9008091EC0081608093EC0013312C
:1007B00011F4988401C099848090A6017090A701DB
:1007C000C12CD12C5E01EAE0AE0EB11CE12CF12C63
:1007D00088E0682E5524539477C0F50101915F019C
:1007E0009B818091A501882369F0C65FDE4F9883C5
:1007F000CA50D1407BD41092A501C65FDE4F9881CC
:10080000CA50D1408D81C65FDE4F9883CA50D14017
:1008100052DF8091A7014FDF8091A6014CDF802F2E
:100820004ADFC65FDE4F9881CA50D140133119F4B8
:100830002D8126252D83E114F10479F4091569F041
:100840008F81C0FE04C0133111F4886001C0877F1E
:100850008F83E090A601F090A70190FD11C0E114F4
:10086000F10421F493FD02C0997F92600F812C81E5
:10087000492DB701892F43D481112DC0E12CF12CD2
:10088000C0FC02C01531E9F48091A6019091A70146
:10089000A091A801B091A9010196A11DB11D80935D
:1008A000A6019093A701A093A801B093A9011331C9
:1008B00041F4AA27BB27892B8A2B8B2B11F450924A
:1008C000A501FFEFCF1ADF0A89819A81C816D906E0
:1008D00008F483CF80E09B8197FF2AC08E81EBDEF6
:1008E000872DE9DE882DE7DE80E0E5DE8B8185FF60
:1008F00006C0E114F10419F48F7C80618B830F81B1
:100900002C81492DB7018B81FAD3133189F44091A1
:10091000A6015091A7016091A8017091A9016627D5
:100920007727452B462B472B19F491E09093A5018F
:100930001093F1008093F1008091E8008E7780930E
:10094000E800C65FDE4F0FB6F894DEBF0FBECDBF26
:10095000DF91CF911F910F91FF90EF90DF90CF909B
:10096000BF90AF909F908F907F906F905F90089511
:10097000DF92EF92FF920F931F93CF93DF9300D0FC
:100980001F92CDB7DEB7F82E40E050E063E070E094
:10099000CE0101960E94C80F89819A8199838A832A
:1009A0008091E8008B778093E80083E08093E900F2
:1009B0008091EC0081608093EC00F092F100109245
:1009C000F10000E010E098E0E92EDD24D39449C066
:1009D0008091A501882319F089D31092A5018B81FC
:1009E0006ADE8091A70167DE8091A60164DE78DE71
:1009F0008093F1008091E80085FD07C08091E800B8
:100A00008E778093E8000E94CA1184E1F81203C037
:100A10008B818E258B8300FD03C086E1F8121FC0F9
:100A20004091A6015091A7016091A8017091A90180
:100A30004F5F5F4F6F4F7F4F4093A6015093A701C9
:100A40006093A8017093A90186E1F81641F066272A
:100A50007727452B462B472B11F4D092A5010F5F2A
:100A60001F4F29813A810217130708F4B1CF109262
:100A7000F1009091E8008091E8008E778093E80083
:100A800095FD09C00E94CA118091E8008E7780937D
:100A9000E8000E94CA110F900F900F90DF91CF9144
:100AA0001F910F91FF90EF90DF900895BF92CF922A
:100AB000DF92EF92FF920F931F93CF93DF93CDB707
:100AC000DEB729970FB6F894DEBF0FBECDBFB82EA4
:100AD00040E050E065E070E0CE0101960E94C80F52
:100AE0009091E8009B779093E80083E08093E90081
:100AF0009091EC0091609093EC008E010E5F1F4F7F
:100B00007E0186E0E80EF11C6701F80181918F01FA
:100B1000DCDDF70181937F010C151D05B1F7B09263
:100B2000F1001092F1008981FE01E80FF11D85812D
:100B30008093F1001092F1008091E8008E7780930D
:100B4000E80029960FB6F894DEBF0FBECDBFDF9147
:100B5000CF911F910F91FF90EF90DF90CF90BF90BA
:100B60000895DF92EF92FF920F931F93CF93DF933D
:100B700000D000D0CDB7DEB7D82E40E050E064E022
:100B800070E0CE0101960E94C80F9091E8009B771B
:100B90009093E80083E08093E9009091EC009160ED
:100BA0009093EC008E010F5F1F4F7E0185E0E80EF1
:100BB000F11CF80181918F017EDD0E151F05C9F72B
:100BC000D092F1001092F1001092F1008091E800B3
:100BD0008E778093E8000F900F900F900F90DF9129
:100BE000CF911F910F91FF90EF90DF900895FF92AA
:100BF0000F931F93CF93DF93CDB7DEB7C250D14091
:100C00000FB6F894DEBF0FBECDBF40E050E063E00A
:100C100070E0CE0101960E94C80F69818E010C5FC1
:100C20001F4F40E050E070E0C8010E94C80F809163
:100C3000E8008B778093E80083E08093E90080915F
:100C4000EC0081608093EC008DE18093F1001092C4
:100C5000F100F12C0BC08981F81628F4F801EF0D92
:100C6000F11D808101C080E026DDF3948B81F816B0
:100C700090F310E01CC08981F81650F4E4E0F0E035
:100C8000EC0FFD1FEF0DF11DF39480811EDD01C0FF
:100C900027DD8093F1008091E80085FD07C08091F9
:100CA000E8008E778093E8000E94CA111F5F8A8156
:100CB000181708F31092F1009091E8008091E80075
:100CC0008E778093E80095FD09C00E94CA1180913B
:100CD000E8008E778093E8000E94CA11CE5FDE4F55
:100CE0000FB6F894DEBF0FBECDBFDF91CF911F913D
:100CF0000F91FF90089506C0EFE9FFE03197F1F7FB
:100D000000C00000882321F09AB581509111F4CFE2
:100D10000895EF92FF920F931F93CF93DF9300D02C
:100D200000D000D0CDB7DEB740E050E066E070E024
:100D3000CE0101960E94C80F8091E8008B778093C6
:100D4000E80083E08093E9008091EC00816080936B
:100D5000EC008E010D5F1F4F7E0187E0E80EF11C55
:100D6000F80181918F01A7DC0E151F05C9F78A8153
:100D7000811104C08981BFDF80E001C099D192E177
:100D80009093F1008093F1008091E8008E7780933A
:100D9000E80026960FB6F894DEBF0FBECDBFDF91F8
:100DA000CF911F910F91FF90EF9008950F931F9394
:100DB000CF93DF9300D0CDB7DEB740E050E062E0E4
:100DC00070E0CE0101960E94C80F08EE10E0F80115
:100DD00080818B77808383E08093E900ECEEF0E004
:100DE000808181608083898186DF80E055D1D8D081
:100DF0008A8181DFE1EFF0E081E180831082F801F8
:100E000080818E7780830F900F90DF91CF911F911B
:100E10000F910895CF92DF92EF92FF920F931F935D
:100E2000CF93DF93CDB7DEB72F970FB6F894DEBF21
:100E30000FBECDBF40E050E06BE070E0CE01019608
:100E40000E94C80F8091E8008B778093E80083E0D0
:100E50008093E9008091EC0081608093EC00109217
:100E6000A6011092A7011092A8011092A9018B81EE
:100E700042DFC2D081E010D18A813DDF7E018CE06B
:100E8000E80EF11C23C08D8136DFF80181918F01BE
:100E90001CDCF60181936F010E151F05A1F78F81F0
:100EA000882351F0EBE0F0E0EC0FFD1FE80FF11D9F
:100EB00090818E81981302C080E017C080E0ECD052
:100EC0008A8119DF81E0E8D08A8115DF8C81982F33
:100ED00091509C83882341F08AB5882329F08E01A4
:100EE000085F1F4F6701CFCF80EC90E19093F10036
:100EF0008093F1008091E8008E778093E8002F9630
:100F00000FB6F894DEBF0FBECDBFDF91CF911F911A
:100F10000F91FF90EF90DF90CF9008951F920F9266
:100F20000FB60F9211248F93199908C08091A301D5
:100F300087FF02C02A9A19C02A9817C08091A3017E
:100F4000880F8093A3018091A20181508093A20118
:100F5000811104C01092810082E086BB1B9B05C0FA
:100F60008091A30181608093A301199A8F910F90C2
:100F70000FBE0F901F9018953E9A10926F0010921E
:100F800085001092840081E090E090938900809326
:100F9000880080E48093800089E080938100089538
:100FA00080915C01882349F084B1897F84B985B13F
:100FB000867F85B91CBC1DBC089584B1897F84B926
:100FC00085B1867F85B9D8CF92E090936F0010925B
:100FD000850010928400E82FF0E0EE0FFF1FE5552A
:100FE000FF4F85919491909389008093880010928F
:100FF000800010928100089588E933DB8730D0F4B7
:1010000091E090935C01E82FF0E0EE54FF4FE49103
:10101000209A289A84B1866084B923982B9A8DB53A
:10102000E6FF02C0816001C08E7F8DBD2098E06523
:10103000ECBD089510925C0194B1966094B995B19D
:10104000996095B9C1CF8093A30188E08093A201F4
:101050008091A30187FF02C02A9A01C02A981092AA
:101060008500109284008AE0809381008091A20123
:10107000882319F08AB58111F9CF109281008091EF
:10108000A301089590915C01992329F08EBD0DB4C0
:1010900007FEFDCF0895D7CF882339F0249A8EE933
:1010A000E0DA811103C02C9A089524982C980895B1
:1010B00080EFE8DF80E0E6DF80E0E4DF80915C0144
:1010C000882331F01EBC0DB407FEFDCF8EB502C0E3
:1010D00080E0B9DF80FF03C08AB58111E9CF8AB50E
:1010E000882311F080E0089581E808958DE4CADF37
:1010F00080E0C8DF8091A801C5DF80E0C3CF0F93F7
:101100001F93CF93DF93EB01142F8E77E82FF0E03E
:10111000E830F10569F134F4E230F10559F0349723
:1011200049F50BC0E032F10541F0E034F10501F181
:10113000709701F5822FDFDD1DC0802FA3DF8D2F7B
:10114000A1DF8C2F9FDF80915C01882331F01EBCD2
:101150000DB407FEFDCF8EB502C080E074DF8113B1
:1011600003C08AB58111E9CF8AB5882329F002C06E
:101170009FDF03C080E001C080E894E69ABDDF9164
:10118000CF911F910F9108959B01692F782F832F85
:10119000922F0895CF93DF93CDB7DEB7C750D140DC
:1011A0000FB6F894DEBF0FBECDBF40E050E067E061
:1011B00070E0CE018F5F9E4FEBD6CE5FDE4F688131
:1011C00079818A819B81C250D140DEDFCE5FDE4FC4
:1011D000688379838A839B83C250D140CA5FDE4F84
:1011E0008881C650D140C95FDE4F9881C750D14039
:1011F000CA5FDE4F9883C650D140C95FDE4F8883F7
:10120000C750D1408091E8008B778093E80083E05D
:101210008093E9008091EC0081608093EC008091E4
:10122000A401CA5FDE4F28813981C650D1408111A7
:1012300012C0CE5FDE4F688179818A819B81C25066
:10124000D140AE014F5F5F4FE5D3882311F080E0BE
:101250000EC083E00CC0A901BE016F5F7F4FCE5F5F
:10126000DE4F88819981C250D140C3D5EECF90E541
:101270009093F10095E09093F1008093F10081113B
:101280000BC0CA5FDE4F68817981C650D14040E013
:1012900050E0CE0101962ED68091E8008E778093A3
:1012A000E800C95FDE4F0FB6F894DEBF0FBECDBFBA
:1012B000DF91CF910895AF92BF92CF92DF92EF92DC
:1012C000FF920F931F93CF93DF93CDB7DEB7C85034
:1012D000D1400FB6F894DEBF0FBECDBF40E050E066
:1012E00068E070E0CE01019653D66B817C818D81E0
:1012F0009E814ADF6B837C838D839E837F8168859B
:101300006F83788740E050E0CE01099641D68F8107
:10131000988509968F739927892B39F48091E80075
:101320008B778093E8000E94CA118091E8008B7748
:101330008093E80083E08093E9008091EC00816075
:101340008093EC008091A40181112EC0298121504D
:10135000EB80FC800D811E812630A0F430E0F90185
:10136000E359FE4F8081F901ED58FE4F9081F9015C
:10137000E758FE4F6081F901E158FE4F208122239A
:1013800059F103C066E293E28EE2AF80B88429E0AF
:10139000C22ED12CCC0EDD1E2A81482F892FA2D33C
:1013A00081110BC083E00AC04F815885BE01675F81
:1013B0007F4F8B819C8149D5F3CF80E090E590935E
:1013C000F10094E09093F1008093F1008091E800A7
:1013D0008E778093E80005C02985B801A70154D312
:1013E000DFCFC85FDE4F0FB6F894DEBF0FBECDBFB4
:1013F000DF91CF911F910F91FF90EF90DF90CF90F1
:10140000BF90AF900895CF93DF931F92CDB7DEB713
:1014100040E050E061E070E0CE010196B9D58091E6
:10142000E8008B778093E80083E08093E900809167
:10143000EC0081608093EC0089818093A40181E5B8
:101440008093F1008981813011F080E001C080EC4F
:101450008093F1008091E8008E778093E8000F90F0
:10146000DF91CF910895CF93DF93CDB7DEB7299762
:101470000FB6F894DEBF0FBECDBF8091F10084306F
:1014800009F493C040F4823079F108F04AC0813009
:1014900009F02CC109C0863009F48BC008F487C05C
:1014A000873009F023C1CEC08091E8008B7780930C
:1014B000E80083E08093E9008091EC0081608093F4
:1014C000EC008091A401811102C01AD205C08230C3
:1014D00011F441D401C080E090E59093F10091E0D7
:1014E0009093F1008927FBC08091E8008B7780936F
:1014F000E80083E08093E9008091EC0081608093B4
:10150000EC008091A401811102C041D201C066D4D7
:1015100080E58093F10082E08093F1001092F10069
:10152000E0C040E050E065E070E0CE01019630D5CB
:101530006A817B818C819D8127DE6A837B838C839A
:101540009D838091E8008B778093E80083E080930F
:10155000E9008091EC0081608093EC008091A4010F
:10156000E981811114C0E150E83028F4F0E0EB5932
:10157000FE4F808101C080E04A815B816C817D816A
:1015800026D3882311F080E00BC083E009C0E1304E
:1015900011F480E101C084E16A817B818ED4F1CFB6
:1015A00090E59093F10093E098C085DE9FC0F2DD56
:1015B0009DC040E050E061E070E0CE010196E8D4CB
:1015C0008091E8008B778093E80083E08093E900C6
:1015D0008091EC0081608093EC008091A4018111E6
:1015E00012C0E981E150E23028F4F0E0EB57FE4F01
:1015F000808101C088E7BE016A5F7F4FD3D1882315
:1016000021F080E003C081E001C083E090E5909389
:10161000F10096E09093F1008093F100811161C098
:101620008E819F81A885B985CD01AA27BB2780938C
:10163000F1008E819F81A885B9858093F100892F63
:1016400099274DC08091F100833029F128F4813031
:1016500041F0823081F516C0843011F1853059F5A2
:1016600024C08091F1009091F1002091F10030911F
:10167000F1003093610120936201909363018093A4
:10168000640117C08091F1009091F10090935F0187
:10169000809360010EC08091F10080935E0109C0CB
:1016A0008091F10080935D0104C08091F1008091F0
:1016B000F10080E001C081E09091E8009B77909379
:1016C000E80093E09093E9009091EC009160909392
:1016D000EC0090E59093F10097E09093F1008093F7
:1016E000F1008091E8008E778093E80029960FB68C
:1016F000F894DEBF0FBECDBFDF91CF9108954D9915
:10170000FECF4D9BFECF4D99FECF5B9A539A8091B1
:10171000C9008F7E8093C9008091C9008860809342
:10172000C90081E08093AA0108958091C80086FFD6
:10173000FCCF8091C80080648093C8008091C9006C
:10174000877F8093C9008091C90080618093C90020
:1017500053985B981092AA0108958091AA01811173
:10176000E4DF80EC8093C8001092C9001092CA0098
:101770008AB1877D8AB98BB1837D8BB908958091B9
:10178000AA018111D2DF8091C800806C8093C800CB
:101790001092C9001092CA008AB1877D8AB98BB1B4
:1017A000837D8BB924982C980895CF93DF931F9253
:1017B000CDB7DEB79091AA01911103C089839FDF55
:1017C00089819091C80095FFFCCF9091C8009064EA
:1017D0009093C8008093CE000F90DF91CF91089531
:1017E0008091AA018111A1DF8091C80087FD03C00B
:1017F0008AB58111F9CF8091CE0008958091AA0118
:10180000811101C07CDF8CE04D99FECF4D9BFECF56
:101810004D99FECF8150C1F708951092AA01249AE4
:101820002C9885E08A95F1F700008AB188628AB920
:1018300052988FE190E09093CD008093CC0088E0A7
:101840008093C9008FE68093CA00D8DFD7CF10926B
:10185000AA018AB188628AB952985B9A85E08A9512
:10186000F1F700008FE190E09093CD008093CC00E1
:1018700088E08093C9008FE68093CA00BFDFBECFA7
:101880001F93CF93DF9300D0CDB7DEB7182F862FED
:1018900079839A838ADF7981872F87DF812F85DF9C
:1018A0009A81892F0F900F90DF91CF911F917DCF5B
:1018B00040916101509162016091630170916401F6
:1018C000482BCB01BA01DCCF80E86FDF89DF9AB506
:1018D000992321F081FFF8CF81E0089580E00895F9
:1018E0008BE663DF8FE0E4DF80E25FDF79DF9AB5CC
:1018F000992321F087FDF8CF81E0089580E00895D5
:10190000BF92CF92DF92EF92FF920F931F93CF93EC
:10191000DF93CDB7DEB728970FB6F894DEBF0FBEC2
:10192000CDBF95DF81EC41DF89E53FDF82EC3DDF14
:1019300082E03BDF80EE39DF7E0189E0E80EF11CBA
:101940008E010F5F1F4F88E0D82EB02EC12EE7E822
:10195000F1E0AB2DBC2D8D2D01900D928A95E1F714
:10196000F70182917F0121DFE016F10681F72896C9
:101970000FB6F894DEBF0FBECDBFDF91CF911F91A0
:101980000F91FF90EF90DF90CF90BF909DCF9CDFA5
:1019900081EC0BDF80E009DF81E807DF21DF8111C7
:1019A000F7CFDBCE1F93CF93DF93182FEB01188275
:1019B00019821A821B8294DF811101C026C08CE437
:1019C000F4DE8AE075DF812FF0DE8CE4EEDE8BE062
:1019D0006FDF81E0EADE78DF8823B9F081DF8823DA
:1019E000A1F08BE6E2DE84E063DF80EADEDE82E007
:1019F000DCDE84E2DADEF4DE8883F2DE8983F0DE88
:101A00008A839AB581E0911101C080E0DF91CF9186
:101A10001F910895CF92DF92EF92FF920F931F9341
:101A2000CF93DF936B017C01EA01890159DF8823A1
:101A300009F18CE4BADE8AE03BDF83E4B6DE8BE6B4
:101A4000B4DEC701B6011CDF80EAAFDE802F815013
:101A5000ACDE84E2AADE0C0F1D1F02C0C1DE89933A
:101A6000C017D10719F08AB58111F8CF9AB581E076
:101A7000911101C080E0DF91CF911F910F91FF90F4
:101A8000EF90DF90CF9008950F931F93CF93DF9344
:101A900000D000D0CDB7DEB7182F022F49835A836C
:101AA0006B837C831DDF882399F08CE47EDE8AE0E3
:101AB000FFDE812F7ADE8CE478DE49815A816B81EA
:101AC0007C81CB01BA01DCDE802F6FDE81E001C0BA
:101AD00080E00F900F900F900F90DF91CF911F91AA
:101AE0000F9108952F923F924F925F926F927F9243
:101AF0008F929F92AF92BF92CF92DF92EF92FF921E
:101B00000F931F93CF93DF93782E662E842E922E01
:101B100017012801E60120FF11C0E2DE811102C099
:101B200080E042C08CE441DE8AE0C2DE862D3DDEEC
:101B30008CE43BDE8BE0BCDE81E037DEA114B10437
:101B400019F491FC1FC02FC0CBDE882349F38CE42D
:101B50002CDE8AE0ADDE872D28DE8BE626DEC20194
:101B6000B1018EDE80EA21DE8A2D81501EDE84E600
:101B70001CDEAC0EBD1E02C0899117DECA15DB0546
:101B8000D9F7DFCFADDE882309F4CACF8CE40DDEB0
:101B90008AE08EDE882D09DE8CE407DEC201B10109
:101BA0006FDE80E002DE81E0DF91CF911F910F9127
:101BB000FF90EF90DF90CF90BF90AF909F908F906D
:101BC0007F906F905F904F903F902F9008951F935C
:101BD000CF93DF9300D000D0CDB7DEB7182F498365
:101BE0005A836B837C837CDE49815A816B817C8143
:101BF000882309F467C08CE4103429F4D6DD8AE028
:101C000057DE80E440C049835A836B837C83103362
:101C100009F040C0CADD8AE04BDE86E3C6DD8CE415
:101C2000C4DD8BE045DE81E0C0DD5ADE882309F4A7
:101C300049C08CE4BADD8AE03BDE83E3B6DD8BE6A7
:101C4000B4DD49815A816B817C81CB01BA0118DEF8
:101C500080EAABDD80915F018150A7DD84E6A5DDE0
:101C600010E003C080E0A1DD1F5F212F30E08091F4
:101C70005F019091600128173907A0F38CE495DD8E
:101C80008AE016DE80E391DD8CE48FDD8BE010DEF0
:101C900081E00FC08ADD8AE00BDE812F86DD8CE4D7
:101CA00084DD49815A816B817C81CB01BA01E8DDF9
:101CB00080E07BDD0F900F900F900F90DF91CF9120
:101CC0001F9102CE80E00F900F900F900F90DF9148
:101CD000CF911F910895282F207330E0220F331FDA
:101CE00020693F6F8F70822B60CD1F93CF93DF935E
:101CF0001F92CDB7DEB7182F88E6998356DD812F66
:101D000054DD89E652DD9981892F0F90DF91CF91C3
:101D10001F914BCD80E849DD63DD9AB5992321F011
:101D200081FFF8CF81E0089580E0089580915D0102
:101D3000282F207330E0220F331F20618F70822BF9
:101D400034DD4EDD9AB5992321F087FDEFCF81E098
:101D5000089580E00895BF92CF92DF92EF92FF92B4
:101D60000F931F93CF93DF93CDB7DEB728970FB6AE
:101D7000F894DEBF0FBECDBF50DD82EC16DD82E0F1
:101D800014DD80EE12DD7E0189E0E80EF11C8E018B
:101D90000F5F1F4F58E0D52EB02EC12EEFE8F1E0B7
:101DA000AB2DBC2D8D2D01900D928A95E1F7F70199
:101DB00082917F01FADCE016F10681F728960FB6D2
:101DC000F894DEBF0FBECDBFDF91CF911F910F9171
:101DD000FF90EF90DF90CF90BF909CCF9BDF80EC87
:101DE000E4DC80E0E2DC81E8E0DCFADC8111F7CFC2
:101DF000C6CCEF92FF920F931F93CF93DF937C019A
:101E0000EB018A0193DF8823C1F080915E0163DFDB
:101E100080E0CBDCC70169DF0C0F1D1F04C084E22A
:101E2000C4DCDEDC8993C017D10719F08AB58111B3
:101E3000F6CF9AB581E0911101C080E0DF91CF919A
:101E40001F910F91FF90EF900895EF92FF920F93E3
:101E50001F93CF93DF937C018B01EA0167DF811130
:101E600002C080E023C0C0FF06C0F801EC0FFD1FD8
:101E70008FEF8083219680915E012DDF8DE195DCCF
:101E8000C70133DF10C052DF882359F384E68DDCAD
:101E9000F80180818ADC84E688DCF80181810E5FAC
:101EA0001F4F83DC2297209771F781E0DF91CF915C
:101EB0001F910F91FF90EF9008951F93CF93DF93A1
:101EC000182FEB0133DF882381F080915E0103DF5F
:101ED000812F6BDCCE01816008DF80E666DC80E06C
:101EE00064DCDF91CF911F9121CF80E0DF91CF9112
:101EF0001F910895BF92CF92DF92EF92FF920F93BE
:101F00001F93CF93DF937C018B01EA0143D2B82E5C
:101F1000811133C0209731F028813981021B130BC6
:101F2000E20EF31EC12CD12C23C08091E80085FD68
:101F300015C08091E8008E778093E80056D42097F2
:101F400049F0888199818C0D9D1D9983888325E0B6
:101F5000B22E13C01FD2882359F00EC0F701819111
:101F60007F018093F10001501109FFEFCF1ADF0AC2
:101F700001151105D1F601C0B82E8B2DDF91CF913F
:101F80001F910F91FF90EF90DF90CF90BF90089539
:101F9000BF92CF92DF92EF92FF920F931F93CF9356
:101FA000DF937C018B01EA01F5D1B82E811133C09A
:101FB000209731F028813981021B130BE20EF31EAA
:101FC000C12CD12C23C08091E80085FD15C08091E3
:101FD000E8008B778093E80008D4209749F0888147
:101FE00099818C0D9D1D9983888345E0B42E13C083
:101FF000D1D1882359F00EC08091F100F70181936F
:102000007F0101501109FFEFCF1ADF0A01151105F9
:10201000D1F601C0B82E8B2DDF91CF911F910F917A
:10202000FF90EF90DF90CF90BF900895BF92CF9236
:10203000DF92EF92FF920F931F93CF93DF936C0188
:102040008B017A01A7D1B82E81113AC0E8012197FE
:10205000CC0DDD1DE114F10439F0F701208131814F
:10206000021B130BC21BD30BC12CD12C24C080919B
:10207000E80085FD17C08091E8008B778093E80029
:10208000B4D3E114F10451F0F701808191818C0DFA
:102090009D1D9183808355E0B52E12C07BD188238E
:1020A00051F00DC08091F1008883219701501109F2
:1020B000FFEFCF1ADF0A01151105C9F601C0B82ECE
:1020C0008B2DDF91CF911F910F91FF90EF90DF90BB
:1020D000CF90BF9008952091B3013091B40126179D
:1020E000370748F06115710539F42091E8002E7723
:1020F0002093E80001C0B9019C0180E033C09EB389
:10210000992309F442C0953009F441C09091E80048
:1021100093FD39C09091E80092FD2FC09091E800A6
:1021200090FF20C08091F20090E0F901821B930B98
:1021300005C021912093F100615071099F01280F82
:10214000391F6115710519F02031310590F381E0D7
:102150002031310509F080E09091E8009E7790935E
:10216000E8009F016115710551F68111C8CF05C0C6
:102170008EB3882351F0853051F08091E80082FFC2
:10218000F7CF80E0089581E0089582E0089583E02C
:1021900008952091B3013091B4012617370748F014
:1021A0006115710539F42091E8002E772093E8003D
:1021B00001C0B9019C0180E034C09EB3992309F4A9
:1021C00043C0953009F442C09091E80093FD3AC0B5
:1021D0009091E80092FD30C09091E80090FF21C0FE
:1021E0008091F20090E0F901821B930B06C02491CC
:1021F0002093F1003196615071099C012E0F3F1F11
:102200006115710519F02031310588F381E0203125
:10221000310509F080E09091E8009E779093E80006
:102220009F016115710549F68111C7CF05C08EB3B5
:10223000882351F0853051F08091E80082FFF7CF7C
:1022400080E0089581E0089582E0089583E0089594
:10225000EF92FF920F931F93CF93DF938B01209107
:10226000B3013091B4012617370748F061157105A5
:1022700039F42091E8002E772093E80001C089010D
:10228000382F492F20E036C08EB3882309F445C08B
:10229000853009F444C08091E80083FD3CC0809102
:1022A000E80082FD32C08091E80080FF23C0E0900A
:1022B000F200F12CC32FD42FEC1AFD0A07C0CE0177
:1022C000AFD28093F100219601501109CE018E0DFD
:1022D0009F1D0115110519F08031910580F321E052
:1022E000409709F020E08091E8008E778093E80025
:1022F0003C2F4D2F0115110539F62111C5CF05C011
:102300008EB3882351F0853051F08091E80082FF30
:10231000F7CF80E005C081E003C082E001C083E028
:10232000DF91CF911F910F91FF90EF9008958F70E3
:102330008093E900EBEEF0E0808181608083EDEE38
:10234000F0E010826093EC0040838091EE00881FE3
:102350008827881F08958091AD0187FD05C0809171
:10236000E80080FF0DC010C08091E80082FD04C02D
:102370008EB38111F9CF08958091E8008B7707C063
:102380008EB38111ECCF08958091E8008E77809311
:10239000E80008958091E4009091E50045E62091E1
:1023A000EC0020FD1EC022C02EB3222391F0253068
:1023B00091F02091EB0025FD10C02091E4003091B8
:1023C000E5002817390759F34150C90141F784E066
:1023D000089582E0089583E0089581E0089580E003
:1023E00008952091E80020FFDFCFF9CF2091E80089
:1023F00022FFDACFF4CF3CD03ED08091D8008F7747
:102400008093D8008091D80080688093D800809114
:10241000D8008F7D8093D80084E089BD86E089BD97
:1024200009B400FEFDCF1EBA1092AB0142E160E09C
:1024300080E07DDF8091E1008E7F8093E1008091DC
:10244000E20081608093E2008091E20088608093E6
:10245000E2008091E0008E7F8093E0000895E3E643
:10246000F0E080818E7F808381E08093AC01C3CFD8
:102470001092E20008951092E10008951F920F92C9
:102480000FB60F9211242F933F934F935F936F9347
:102490007F938F939F93AF93BF93EF93FF9380911D
:1024A000E10080FF17C08091E20080FF13C080919F
:1024B000E2008E7F8093E2008091E2008061809351
:1024C000E2008091D80080628093D80019BC1EBAC7
:1024D0000E943A018091E10084FF2FC08091E200C8
:1024E00084FF2BC084E089BD86E089BD09B400FE6D
:1024F000FDCF8091D8008F7D8093D8008091E1003E
:102500008F7E8093E1008091E2008F7E8093E200D5
:102510008091E20081608093E2008091AB0188238A
:1025200011F084E007C08091E30087FF02C083E0E0
:1025300001C081E08EBB0E9438018091E10083FFE1
:1025400021C08091E20083FF1DC08091E100877F60
:102550008093E10082E08EBB1092AB018091E1009C
:102560008E7F8093E1008091E2008E7F8093E20075
:102570008091E20080618093E20042E160E080E0CF
:10258000D6DE32D1FF91EF91BF91AF919F918F91A4
:102590007F916F915F914F913F912F910F900FBE5F
:1025A0000F901F9018951F93CF93DF9300D01F9229
:1025B000CDB7DEB7EDEAF1E08091F100819381E0E3
:1025C000E53BF807C9F710D18091E80083FFF7C019
:1025D0008091AD019091AE01953009F470C038F44E
:1025E000913079F170F0933009F0E9C02AC0983049
:1025F00009F4B7C0993009F4C6C0963009F0DFC0BD
:1026000083C0803899F0823809F0D9C08091B10137
:102610009091B2018F7099278093E9009091EB001F
:1026200095FB992790F91092E90001C090E0809104
:10263000E800877F8093E8009093F1001092F1000A
:102640009BC0882319F0823009F0B9C08F718230A5
:1026500009F0B5C08091AF0181112BC08091B1010B
:102660009091B2018F709927009709F4A8C08093C8
:10267000E9002091EB0020FF1CC02091AE01233027
:1026800021F48091EB00806212C09091EB00906188
:102690009093EB0021E030E001C0220F8A95EAF729
:1026A0002093EA001092EA008091EB00886080930A
:1026B000EB001092E9008091E800877F60C08111F3
:1026C0007EC08091AF019091B0018F779927182F2C
:1026D0009091E3009078982B9093E3008091E8002C
:1026E000877F8093E80037DE8091E80080FFFCCF91
:1026F0008091E30080688093E300112311F083E070
:1027000001C082E08EBB5BC08058823008F057C0A9
:102710009E012D5F3F4FAE014F5F5F4F6091B10152
:102720008091AF019091B0010E947401BC010097AB
:1027300009F445C08091E800877F8093E8002B81F1
:1027400089819A81211102C024DD05C0213011F454
:102750007FDD01C0C0DC8091E8008B778093E800CA
:102760002EC0803861F58091E800877F8093E80073
:102770008091AB018093F1008091E8008E77809387
:10278000E800E9DD1CC081111AC09091AF019230C0
:10279000B0F48091E800877F8093E8009093AB01CC
:1027A000DADD8091AB01811104C08091E30087FFE5
:1027B00002C084E001C081E08EBB0E943C01809198
:1027C000E80083FF0AC08091E800877F8093E800DB
:1027D0008091EB0080628093EB000F900F900F9040
:1027E000DF91CF911F9108950895CF938EB38823E1
:1027F000A9F08091E9008F709091EC0090FF02C0E9
:1028000090E801C090E0C92FC82B1092E900809198
:10281000E80083FDC8DECF70C093E900CF91089532
:10282000F999FECF92BD81BDF89A992780B5089598
:10283000262FF999FECF92BD81BDF89A019700B479
:10284000021639F01FBA20BD0FB6F894FA9AF99A19
:082850000FBE0895F894FFCFBC
:102858001C033000300030003200300030003000FF
:102868003100320033003400350000000000090256
:102878002000010100C0320904000002FF0000002E
:102888000705830240000A0705020240000A80018A
:10289800008101009001009101019201179401212A
:1028A8009803069E0301A10100A40300013233200E
:1028B80000C001000140206830222A3218242C353B
:1028C8004C081A23233323232326263626262601BB
:1028D800010100000138391289AB45CDD888FF12B3
:1028E80089AB45CDD888FF4156524953505F4D4B6F
:0228F8003200AC
:00000001FF
